Archive member included       because of file (symbol)

./libfontprn.a(fontprn.o)     menu.o (FontPrintInit)
./libbg_rsm.a(bgmain.o)       menuitem.o (bgMain)
./libbg_rsm.a(bgexpl.o)       menuitem.o (bg_title_str)
./libbg_rsm.a(bg_map_map.o)   ./libbg_rsm.a(bgmain.o) (map_data_front)
./libbg_rsm.a(ball.o)         ./libbg_rsm.a(bgmain.o) (ball_Palette)
./libbg_rsm.a(bg_map.o)       ./libbg_rsm.a(bgmain.o) (bg_map_Palette)
./libbg_rsm.a(cl0.o)          ./libbg_rsm.a(bgmain.o) (cl0_Palette)
./libbmpmode.a(bitmap.o)      menuitem.o (bm_Main)
./libbmpmode.a(bmexpl.o)      menuitem.o (bm_title_str)
./libbmpmode.a(img24bit.o)    ./libbmpmode.a(bitmap.o) (img24bit_RawBitmap)
./libbmpmode.a(img24bit2.o)   ./libbmpmode.a(bitmap.o) (img24bit2_RawBitmap)
./libbmpmode.a(umiB.o)        ./libbmpmode.a(bitmap.o) (umiB_Palette)
./libcoleffsm.a(c_effect.o)   menuitem.o (ceMain)
./libcoleffsm.a(ce_data.o)    ./libcoleffsm.a(c_effect.o) (ce_OamData_Sample)
./libcoleffsm.a(ceexpl.o)     menuitem.o (ce_title_str)
./libcoleffsm.a(ce_PS_hey5.o)
                              ./libcoleffsm.a(c_effect.o) (ce_PS_hey5_Palette)
./libcoleffsm.a(ce_bg1.o)     ./libcoleffsm.a(c_effect.o) (ce_bg1_Palette)
./libcoleffsm.a(ce_bg3.o)     ./libcoleffsm.a(c_effect.o) (ce_bg3_Character)
./libalphasm.a(alpha.o)       menuitem.o (apMain)
./libalphasm.a(alpha_data.o)  ./libalphasm.a(alpha.o) (ap_OamData_Sample)
./libalphasm.a(alexpl.o)      menuitem.o (ap_title_str)
./libalphasm.a(ap_bg0.o)      ./libalphasm.a(alpha.o) (ap_bg0_Palette)
./libalphasm.a(ap_bg1.o)      ./libalphasm.a(alpha.o) (ap_bg1_Character)
./libalphasm.a(ap_bg2.o)      ./libalphasm.a(alpha.o) (ap_bg2_Character)
./libalphasm.a(ap_PS_hey5.o)  ./libalphasm.a(alpha.o) (ap_PS_hey5_Palette)
./libobj_rsm.a(obmain.o)      menuitem.o (obMain)
./libobj_rsm.a(obexpl.o)      menuitem.o (ob_title_str)
./libobj_rsm.a(hey2.o)        ./libobj_rsm.a(obmain.o) (hey2_Palette)
./libswinsm.a(window.o)       menuitem.o (swMain)
./libswinsm.a(swexpl.o)       menuitem.o (sw_title_str)
./libswinsm.a(sw_bg1.o)       ./libswinsm.a(window.o) (sw_bg1_Character)
./libswinsm.a(sw_bg2.o)       ./libswinsm.a(window.o) (sw_bg2_Character)
./libswinsm.a(sw_bg3.o)       ./libswinsm.a(window.o) (sw_bg3_Character)
./libswinsm.a(sw_bg0.o)       ./libswinsm.a(window.o) (sw_bg0_Palette)
./libswinsm.a(sw_PS_hey5.o)   ./libswinsm.a(window.o) (sw_PS_hey5_Palette)
C:\PROGRA~1\CYGNUS\THUMBELF-000512\H-I686-CYGWIN32\BIN/../lib/gcc-lib/thumb-elf/2.9-arm-000512/libgcc.a(_call_via_rX.o)
                              main.o (_call_via_r0)
C:\PROGRA~1\CYGNUS\THUMBELF-000512\H-I686-CYGWIN32\BIN/../lib/gcc-lib/thumb-elf/2.9-arm-000512/libgcc.a(_divsi3.o)
                              share.o (__divsi3)
C:\PROGRA~1\CYGNUS\THUMBELF-000512\H-I686-CYGWIN32\BIN/../lib/gcc-lib/thumb-elf/2.9-arm-000512/libgcc.a(_dvmd_tls.o)
                              C:\PROGRA~1\CYGNUS\THUMBELF-000512\H-I686-CYGWIN32\BIN/../lib/gcc-lib/thumb-elf/2.9-arm-000512/libgcc.a(_divsi3.o) (__div0)
C:\PROGRA~1\CYGNUS\THUMBELF-000512\H-I686-CYGWIN32\BIN/../lib/gcc-lib/thumb-elf/2.9-arm-000512/libgcc.a(_udivsi3.o)
                              ./libfontprn.a(fontprn.o) (__udivsi3)
C:\PROGRA~1\CYGNUS\THUMBELF-000512\H-I686-CYGWIN32\BIN/../lib/gcc-lib/thumb-elf/2.9-arm-000512/libgcc.a(_umodsi3.o)
                              ./libfontprn.a(fontprn.o) (__umodsi3)
C:\PROGRA~1\CYGNUS\THUMBELF-000512\H-I686-CYGWIN32\BIN/../lib/gcc-lib/thumb-elf/2.9-arm-000512/../../../../thumb-elf/lib/libg.a(memcpy.o)
                              ./libfontprn.a(fontprn.o) (memcpy)

Allocating common symbols
Common symbol       size              file

ob_pos_y            0x4               ./libobj_rsm.a(obmain.o)
bg2pa               0x4               ./libbmpmode.a(bitmap.o)
ap_eff_type         0x4               ./libalphasm.a(alpha.o)
bg_pa               0x4               ./libbg_rsm.a(bgmain.o)
menu_old_cursor_pos
                    0x4               menu.o
v_blank_fnc         0x4               share.o
bg2pb               0x4               ./libbmpmode.a(bitmap.o)
start_y             0x4               ./libbmpmode.a(bitmap.o)
menu_prev_cursor_pos
                    0x4               menu.o
bg_pos_y            0x4               ./libbg_rsm.a(bgmain.o)
bg_ball_anim_count_change_mode
                    0x4               ./libbg_rsm.a(bgmain.o)
ce_EVY_rate         0x4               ./libcoleffsm.a(c_effect.o)
menu_cursor_pos     0x4               menu.o
bg_start_x          0x4               ./libbg_rsm.a(bgmain.o)
ap_obj_alpha        0x4               ./libalphasm.a(alpha.o)
Cont                0x4               share.o
ob_mosaic           0x4               ./libobj_rsm.a(obmain.o)
ob_affine           0x4               ./libobj_rsm.a(obmain.o)
menu_prev_page      0x4               menu.o
bg_oam_buffer       0x20              ./libbg_rsm.a(bgmain.o)
ce_EVB_rate         0x4               ./libcoleffsm.a(c_effect.o)
bg_rotate           0x4               ./libbg_rsm.a(bgmain.o)
ce_eff_type         0x4               ./libcoleffsm.a(c_effect.o)
bg_pb               0x4               ./libbg_rsm.a(bgmain.o)
ob_pos_x            0x4               ./libobj_rsm.a(obmain.o)
sw_OamBak           0x400             ./libswinsm.a(window.o)
bg_pd               0x4               ./libbg_rsm.a(bgmain.o)
ap_BgBak            0x800             ./libalphasm.a(alpha.o)
Trg                 0x4               share.o
bg_scale_x          0x4               ./libbg_rsm.a(bgmain.o)
start_x             0x4               ./libbmpmode.a(bitmap.o)
bg_ball_anim_count  0x4               ./libbg_rsm.a(bgmain.o)
bg_mosaic           0x4               ./libbg_rsm.a(bgmain.o)
ap_evb              0x4               ./libalphasm.a(alpha.o)
ob_scale_y          0x4               ./libobj_rsm.a(obmain.o)
bg2pd               0x4               ./libbmpmode.a(bitmap.o)
ce_BgBak            0x800             ./libcoleffsm.a(c_effect.o)
bg_pos_x            0x4               ./libbg_rsm.a(bgmain.o)
ce_OamBak           0x400             ./libcoleffsm.a(c_effect.o)
bg_start_y          0x4               ./libbg_rsm.a(bgmain.o)
ob_rotate           0x4               ./libobj_rsm.a(obmain.o)
bg_screen_back_x    0x4               ./libbg_rsm.a(bgmain.o)
IntrMainBuf         0x800             share.o
rotate_value        0x4               ./libbmpmode.a(bitmap.o)
ap_OamBak           0x400             ./libalphasm.a(alpha.o)
menu_page           0x4               menu.o
bg_scale_y          0x4               ./libbg_rsm.a(bgmain.o)
bg2_center_x        0x4               ./libbmpmode.a(bitmap.o)
bg_pc               0x4               ./libbg_rsm.a(bgmain.o)
ce_EVA_rate         0x4               ./libcoleffsm.a(c_effect.o)
IntrCheck           0x4               share.o
ce_obj_mode         0x4               ./libcoleffsm.a(c_effect.o)
Zoom                0x4               ./libbmpmode.a(bitmap.o)
ob_scale_x          0x4               ./libobj_rsm.a(obmain.o)
bg2pc               0x4               ./libbmpmode.a(bitmap.o)
bg2_center_y        0x4               ./libbmpmode.a(bitmap.o)
ap_eva              0x4               ./libalphasm.a(alpha.o)
ob_oam_buffer       0x20              ./libobj_rsm.a(obmain.o)
bm_Bgmode           0x4               ./libbmpmode.a(bitmap.o)

Memory Configuration

Name             Origin             Length             Attributes
*default*        0x00000000         0xffffffff

Linker script and memory map

LOAD crt0.o
LOAD main.o
LOAD share.o
LOAD menu.o
LOAD menuitem.o
LOAD C:/agb/lib/libagbsyscall.a
LOAD C:/agb/lib/libisagbprn.a
LOAD ./libfontprn.a
LOAD ./libbg_rsm.a
LOAD ./libbmpmode.a
LOAD ./libcoleffsm.a
LOAD ./libalphasm.a
LOAD ./libobj_rsm.a
LOAD ./libswinsm.a
LOAD C:\PROGRA~1\CYGNUS\THUMBELF-000512\H-I686-CYGWIN32\BIN/../lib/gcc-lib/thumb-elf/2.9-arm-000512/libgcc.a
LOAD C:\PROGRA~1\CYGNUS\THUMBELF-000512\H-I686-CYGWIN32\BIN/../lib/gcc-lib/thumb-elf/2.9-arm-000512/../../../../thumb-elf/lib/libg.a
LOAD C:\PROGRA~1\CYGNUS\THUMBELF-000512\H-I686-CYGWIN32\BIN/../lib/gcc-lib/thumb-elf/2.9-arm-000512/../../../../thumb-elf/lib/libc.a
LOAD C:\PROGRA~1\CYGNUS\THUMBELF-000512\H-I686-CYGWIN32\BIN/../lib/gcc-lib/thumb-elf/2.9-arm-000512/libgcc.a
Address of section .bss set to 0x3000000
Address of section .text set to 0x8000000
                0x00008000                .=0x8000

.interp
 *(.interp)

.hash
 *(.hash)

.dynsym
 *(.dynsym)

.dynstr
 *(.dynstr)

.gnu.version
 *(.gnu.version)

.gnu.version_d
 *(.gnu.version_d)

.gnu.version_r
 *(.gnu.version_r)

.rel.text
 *(.rel.text)
 *(.rel.text.*)
 *(.rel.gnu.linkonce.t*)

.rela.text
 *(.rela.text)
 *(.rela.text.*)
 *(.rela.gnu.linkonce.t*)

.rel.data
 *(.rel.data)
 *(.rel.data.*)
 *(.rel.gnu.linkonce.d*)

.rela.data
 *(.rela.data)
 *(.rela.data.*)
 *(.rela.gnu.linkonce.d*)

.rel.rodata
 *(.rel.rodata)
 *(.rel.rodata.*)
 *(.rel.gnu.linkonce.r*)

.rela.rodata
 *(.rela.rodata)
 *(.rela.rodata.*)
 *(.rela.gnu.linkonce.r*)

.rel.got
 *(.rel.got)

.rela.got
 *(.rela.got)

.rel.ctors
 *(.rel.ctors)

.rela.ctors
 *(.rela.ctors)

.rel.dtors
 *(.rel.dtors)

.rela.dtors
 *(.rela.dtors)

.rel.init
 *(.rel.init)

.rela.init
 *(.rela.init)

.rel.fini
 *(.rel.fini)

.rela.fini
 *(.rela.fini)

.rel.bss
 *(.rel.bss)

.rela.bss
 *(.rela.bss)

.rel.plt
 *(.rel.plt)

.rela.plt
 *(.rela.plt)

.init
 *(.init)

.plt
 *(.plt)

.text           0x08000000     0x3170
 *(.text)
 .text          0x08000000      0x1cc crt0.o
                0x08000000                _start
                0x080000c0                start_vector
                0x080000fc                intr_main
 .text          0x080001cc       0x60 main.o
                0x080001cc                AgbMain
 .text          0x0800022c      0x25c share.o
                0x08000428                V_Wait
                0x08000448                KeyInit
                0x080002b4                ClearOamRam
                0x08000400                V_Intr_Clear
                0x0800028c                ClearVram
                0x08000414                V_Intr_Set
                0x08000318                ClearPaletteRam
                0x08000388                InitVBlank
                0x0800023c                ClearWorkRam
                0x0800045c                KeyRead
                0x08000340                fix_mul
                0x08000278                ClearGraphicRam
                0x08000358                fix_div
                0x080003c8                SetVBlankFunc
                0x08000370                fix_inverse
                0x080003fc                dummy
                0x0800022c                ClearRamAll
                0x080003e0                VBlankFunc
 .text          0x08000488      0x4fc menu.o
                0x08000488                MenuInit
                0x0800049c                Menu
 .text          0x08000984      0x5e8 ./libfontprn.a(fontprn.o)
                0x08000d64                FontPrintC
                0x08000ad0                FontPrint
                0x08000d88                NumPrintC
                0x08000ac4                FontColor
                0x08000db8                FontPrintCls
                0x08000a84                FontPalletLoad
                0x08000bcc                NumPrint
                0x08000e8c                fp_itoa
                0x08000984                FontPrintInit
                0x08000df0                FontPrintSync
 .text          0x08000f6c      0x69c ./libbg_rsm.a(bgmain.o)
                0x08000f6c                bgMain
 .text          0x08001608      0x36c ./libbmpmode.a(bitmap.o)
                0x08001608                bm_Main
 .text          0x08001974      0x6d0 ./libcoleffsm.a(c_effect.o)
                0x08001d04                ce_v_blank_intr
                0x08001d40                ce_ObjMove
                0x08001974                ceMain
                0x08001fec                ce_moji_pr
                0x08001fa0                ce_suji_pr
 .text          0x08002044      0x64c ./libalphasm.a(alpha.o)
                0x08002044                apMain
                0x080025ec                ap_moji_pr
                0x080023fc                ap_ObjMove
                0x08002644                ap_suji_pr
                0x080023c0                ap_v_blank_intr
 .text          0x08002690      0x4b0 ./libobj_rsm.a(obmain.o)
                0x08002690                obMain
 .text          0x08002b40      0x3c4 ./libswinsm.a(window.o)
                0x08002e34                sw_ObjMove
                0x08002e14                sw_v_blank_intr
                0x08002b40                swMain
 .text          0x08002f04       0x3c C:\PROGRA~1\CYGNUS\THUMBELF-000512\H-I686-CYGWIN32\BIN/../lib/gcc-lib/thumb-elf/2.9-arm-000512/libgcc.a(_call_via_rX.o)
                0x08002f0c                _call_via_r2
                0x08002f1c                _call_via_r6
                0x08002f18                _call_via_r5
                0x08002f10                _call_via_r3
                0x08002f30                _call_via_fp
                0x08002f24                _call_via_r8
                0x08002f20                _call_via_r7
                0x08002f04                _call_via_r0
                0x08002f2c                _call_via_sl
                0x08002f38                _call_via_sp
                0x08002f28                _call_via_r9
                0x08002f14                _call_via_r4
                0x08002f08                _call_via_r1
                0x08002f34                _call_via_ip
                0x08002f3c                _call_via_lr
 .text          0x08002f40       0x94 C:\PROGRA~1\CYGNUS\THUMBELF-000512\H-I686-CYGWIN32\BIN/../lib/gcc-lib/thumb-elf/2.9-arm-000512/libgcc.a(_divsi3.o)
                0x08002f40                __divsi3
 .text          0x08002fd4        0x4 C:\PROGRA~1\CYGNUS\THUMBELF-000512\H-I686-CYGWIN32\BIN/../lib/gcc-lib/thumb-elf/2.9-arm-000512/libgcc.a(_dvmd_tls.o)
                0x08002fd4                __div0
 .text          0x08002fd8       0x78 C:\PROGRA~1\CYGNUS\THUMBELF-000512\H-I686-CYGWIN32\BIN/../lib/gcc-lib/thumb-elf/2.9-arm-000512/libgcc.a(_udivsi3.o)
                0x08002fd8                __udivsi3
 .text          0x08003050       0xc0 C:\PROGRA~1\CYGNUS\THUMBELF-000512\H-I686-CYGWIN32\BIN/../lib/gcc-lib/thumb-elf/2.9-arm-000512/libgcc.a(_umodsi3.o)
                0x08003050                __umodsi3
 .text          0x08003110       0x60 C:\PROGRA~1\CYGNUS\THUMBELF-000512\H-I686-CYGWIN32\BIN/../lib/gcc-lib/thumb-elf/2.9-arm-000512/../../../../thumb-elf/lib/libg.a(memcpy.o)
                0x08003110                memcpy
 *(.text.*)
 *(.stub)
 *(.gnu.warning)
 *(.gnu.linkonce.t*)
 *(.glue_7t)
 *(.glue_7)
                0x08003170                _etext=.
                0x08003170                PROVIDE (etext, .)

.fini
 *(.fini)

.rodata         0x08003170    0x4ed30
 *(.rodata)
 .rodata        0x08003170      0x2b8 share.o
                0x080033f0                IntrTable
                0x08003170                sin_cos_table
 .rodata        0x08003428       0x4c menu.o
 .rodata        0x08003474       0x60 menuitem.o
                0x08003474                mitem
 .rodata        0x080034d4    0x1a428 ./libfontprn.a(fontprn.o)
                0x080034d4                font8
                0x0801d8d4                fontOamData
 .rodata        0x0801d8fc       0xdc ./libbg_rsm.a(bgexpl.o)
 .rodata        0x0801d9d8     0x1000 ./libbg_rsm.a(bg_map_map.o)
                0x0801e1d8                map_data_back
                0x0801d9d8                map_data_front
 .rodata        0x0801e9d8      0x220 ./libbg_rsm.a(ball.o)
                0x0801e9f8                ball_Char
                0x0801e9d8                ball_Palette
 .rodata        0x0801ebf8      0x120 ./libbg_rsm.a(bg_map.o)
                0x0801ebf8                bg_map_Palette
                0x0801ec18                bg_map_Char
 .rodata        0x0801ed18     0x22b4 ./libbg_rsm.a(cl0.o)
                0x0801edca                cl0_Character
                0x0801ed18                cl0_Palette
                0x08020eca                cl0_Map
 .rodata        0x08020fcc       0x9c ./libbmpmode.a(bmexpl.o)
 .rodata        0x08021068    0x12c00 ./libbmpmode.a(img24bit.o)
                0x08021068                img24bit_RawBitmap
 .rodata        0x08033c68     0xa000 ./libbmpmode.a(img24bit2.o)
                0x08033c68                img24bit2_RawBitmap
 .rodata        0x0803dc68     0x9800 ./libbmpmode.a(umiB.o)
                0x0803dc68                umiB_Palette
                0x0803de68                umiB_IndexBitmap
 .rodata        0x08047468       0x34 ./libcoleffsm.a(c_effect.o)
 .rodata        0x0804749c       0x28 ./libcoleffsm.a(ce_data.o)
                0x0804749c                ce_OamData_Sample
 .rodata        0x080474c4       0xf0 ./libcoleffsm.a(ceexpl.o)
 .rodata        0x080475b4      0xa00 ./libcoleffsm.a(ce_PS_hey5.o)
                0x080475b4                ce_PS_hey5_Palette
                0x080477b4                ce_PS_hey5_Char
 .rodata        0x08047fb4     0x13cc ./libcoleffsm.a(ce_bg1.o)
                0x0804807e                ce_bg1_Character
                0x08048e7e                ce_bg1_Map
                0x08047fb4                ce_bg1_Palette
 .rodata        0x08049380     0x298c ./libcoleffsm.a(ce_bg3.o)
                0x0804b80a                ce_bg3_Map
                0x0804944a                ce_bg3_Character
                0x08049380                ce_bg3_Palette
 .rodata        0x0804bd0c       0x58 ./libalphasm.a(alpha.o)
 .rodata        0x0804bd64        0x8 ./libalphasm.a(alpha_data.o)
                0x0804bd64                ap_OamData_Sample
 .rodata        0x0804bd6c       0xd8 ./libalphasm.a(alexpl.o)
 .rodata        0x0804be44      0xc20 ./libalphasm.a(ap_bg0.o)
                0x0804be64                ap_bg0_Character
                0x0804be44                ap_bg0_Palette
                0x0804c564                ap_bg0_Map
 .rodata        0x0804ca64      0xbcc ./libalphasm.a(ap_bg1.o)
                0x0804ca64                ap_bg1_Palette
                0x0804ca6e                ap_bg1_Character
                0x0804d12e                ap_bg1_Map
 .rodata        0x0804d630      0xbcc ./libalphasm.a(ap_bg2.o)
                0x0804d63a                ap_bg2_Character
                0x0804dcfa                ap_bg2_Map
                0x0804d630                ap_bg2_Palette
 .rodata        0x0804e1fc      0xa00 ./libalphasm.a(ap_PS_hey5.o)
                0x0804e1fc                ap_PS_hey5_Palette
                0x0804e3fc                ap_PS_hey5_Char
 .rodata        0x0804ebfc       0xf4 ./libobj_rsm.a(obexpl.o)
 .rodata        0x0804ecf0      0xa00 ./libobj_rsm.a(hey2.o)
                0x0804ecf0                hey2_Palette
                0x0804eef0                hey2_Char
 .rodata        0x0804f6f0        0x8 ./libswinsm.a(window.o)
                0x0804f6f0                sw_OamData_Sample
 .rodata        0x0804f6f8       0x98 ./libswinsm.a(swexpl.o)
 .rodata        0x0804f790      0x694 ./libswinsm.a(sw_bg1.o)
                0x0804f7a4                sw_bg1_Character
                0x0804f924                sw_bg1_Map
                0x0804f790                sw_bg1_Palette
 .rodata        0x0804fe24      0x694 ./libswinsm.a(sw_bg2.o)
                0x0804fe38                sw_bg2_Character
                0x0804ffb8                sw_bg2_Map
                0x0804fe24                sw_bg2_Palette
 .rodata        0x080504b8      0x694 ./libswinsm.a(sw_bg3.o)
                0x080504b8                sw_bg3_Palette
                0x080504cc                sw_bg3_Character
                0x0805064c                sw_bg3_Map
 .rodata        0x08050b4c      0x954 ./libswinsm.a(sw_bg0.o)
                0x08050b4c                sw_bg0_Palette
                0x08050fa0                sw_bg0_Map
                0x08050b60                sw_bg0_Character
 .rodata        0x080514a0      0xa00 ./libswinsm.a(sw_PS_hey5.o)
                0x080514a0                sw_PS_hey5_Palette
                0x080516a0                sw_PS_hey5_Char
 *(.rodata.*)
 *(.gnu.linkonce.r*)

.rodata1
 *(.rodata1)
                0x08051fa0                .=(ALIGN(0x100)+(.&0xff))

.data           0x08051fa0      0x9d8
 *(.data)
 .data          0x08051fa0       0x14 ./libbg_rsm.a(bgexpl.o)
                0x08051fa0                bg_title_str
                0x08051fa8                bg_expl_str_array
                0x08051fa4                bg_expl_str0
 .data          0x08051fb4       0x14 ./libbmpmode.a(bmexpl.o)
                0x08051fb8                bm_expl_str0
                0x08051fbc                bm_expl_str_array
                0x08051fb4                bm_title_str
 .data          0x08051fc8      0x4b0 ./libcoleffsm.a(ce_data.o)
                0x08051fd8                ce_moji_Character
                0x08051fc8                ce_type_tbl
 .data          0x08052478       0x14 ./libcoleffsm.a(ceexpl.o)
                0x0805247c                ce_expl_str0
                0x08052478                ce_title_str
                0x08052480                ce_expl_str_array
 .data          0x0805248c       0x10 ./libalphasm.a(alpha.o)
                0x0805248c                ap_eff_tbl
 .data          0x0805249c      0x4a0 ./libalphasm.a(alpha_data.o)
                0x0805249c                ap_moji_Character
 .data          0x0805293c       0x14 ./libalphasm.a(alexpl.o)
                0x08052944                ap_expl_str_array
                0x0805293c                ap_title_str
                0x08052940                ap_expl_str0
 .data          0x08052950       0x14 ./libobj_rsm.a(obexpl.o)
                0x08052958                ob_expl_str_array
                0x08052950                ob_title_str
                0x08052954                ob_expl_str0
 .data          0x08052964       0x14 ./libswinsm.a(swexpl.o)
                0x08052968                sw_expl_str0
                0x0805296c                sw_expl_str_array
                0x08052964                sw_title_str
 *(.data.*)
 *(.gnu.linkonce.d*)

.data1
 *(.data1)

.ctors
 EXCLUDE_FILE ( *crtend.o )*(.ctors)
 *(SORT(.ctors.*))
 *crtend(.ctors)

.dtors
 EXCLUDE_FILE ( *crtend.o )*(.dtors)
 *(SORT(.dtors.*))
 *crtend.o(.dtors)

.got
 *(.got.plt)
 *(.got)

.dynamic
 *(.dynamic)

.sdata
 *(.sdata)
 *(.sdata.*)
                0x08052978                _edata=.
                0x08052978                PROVIDE (edata, .)
                0x08052978                __bss_start=.
                0x08052978                __bss_start__=.

.sbss
 *(.sbss)
 *(.scommon)

.bss            0x03000000     0x2f20
 *(.dynbss)
 *(.bss)
 .bss           0x03000000      0x9d0 ./libfontprn.a(fontprn.o)
 *(.bss.*)
 *(COMMON)
 COMMON         0x030009d0      0x814 share.o
                                  0x0 (size before relaxing)
                0x030009d0                v_blank_fnc
                0x030009d4                Cont
                0x030009d8                Trg
                0x030009e0                IntrMainBuf
                0x030011e0                IntrCheck
 COMMON         0x030011e4       0x14 menu.o
                                  0x0 (size before relaxing)
                0x030011e4                menu_old_cursor_pos
                0x030011e8                menu_prev_cursor_pos
                0x030011ec                menu_cursor_pos
                0x030011f0                menu_prev_page
                0x030011f4                menu_page
 *fill*         0x030011f8        0x8
 COMMON         0x03001200       0x5c ./libbg_rsm.a(bgmain.o)
                                  0x0 (size before relaxing)
                0x03001200                bg_pa
                0x03001204                bg_pos_y
                0x03001208                bg_ball_anim_count_change_mode
                0x0300120c                bg_start_x
                0x03001210                bg_oam_buffer
                0x03001230                bg_rotate
                0x03001234                bg_pb
                0x03001238                bg_pd
                0x0300123c                bg_scale_x
                0x03001240                bg_ball_anim_count
                0x03001244                bg_mosaic
                0x03001248                bg_pos_x
                0x0300124c                bg_start_y
                0x03001250                bg_screen_back_x
                0x03001254                bg_scale_y
                0x03001258                bg_pc
 COMMON         0x0300125c       0x2c ./libbmpmode.a(bitmap.o)
                                  0x0 (size before relaxing)
                0x0300125c                bg2pa
                0x03001260                bg2pb
                0x03001264                start_y
                0x03001268                start_x
                0x0300126c                bg2pd
                0x03001270                rotate_value
                0x03001274                bg2_center_x
                0x03001278                Zoom
                0x0300127c                bg2pc
                0x03001280                bg2_center_y
                0x03001284                bm_Bgmode
 *fill*         0x03001288        0x8
 COMMON         0x03001290      0xc18 ./libcoleffsm.a(c_effect.o)
                                  0x0 (size before relaxing)
                0x03001290                ce_EVY_rate
                0x03001294                ce_EVB_rate
                0x03001298                ce_eff_type
                0x030012a0                ce_BgBak
                0x03001aa0                ce_OamBak
                0x03001ea0                ce_EVA_rate
                0x03001ea4                ce_obj_mode
 *fill*         0x03001ea8        0x8
 COMMON         0x03001eb0      0xc24 ./libalphasm.a(alpha.o)
                                  0x0 (size before relaxing)
                0x03001eb0                ap_eff_type
                0x03001eb4                ap_obj_alpha
                0x03001ec0                ap_BgBak
                0x030026c0                ap_evb
                0x030026d0                ap_OamBak
                0x03002ad0                ap_eva
 *fill*         0x03002ad4        0xc
 COMMON         0x03002ae0       0x40 ./libobj_rsm.a(obmain.o)
                                  0x0 (size before relaxing)
                0x03002ae0                ob_pos_y
                0x03002ae4                ob_mosaic
                0x03002ae8                ob_affine
                0x03002aec                ob_pos_x
                0x03002af0                ob_scale_y
                0x03002af4                ob_rotate
                0x03002af8                ob_scale_x
                0x03002b00                ob_oam_buffer
 COMMON         0x03002b20      0x400 ./libswinsm.a(window.o)
                                  0x0 (size before relaxing)
                0x03002b20                sw_OamBak
                0x03002f20                .=ALIGN(0x4)
                0x03002f20                .=ALIGN(0x4)
                0x03002f20                _end=.
                0x03002f20                _bss_end__=.
                0x03002f20                __bss_end__=.
                0x03002f20                PROVIDE (end, .)

.stab
 *(.stab)

.stabstr
 *(.stabstr)

.stab.excl
 *(.stab.excl)

.stab.exclstr
 *(.stab.exclstr)

.stab.index
 *(.stab.index)

.stab.indexstr
 *(.stab.indexstr)

.comment
 *(.comment)

.debug
 *(.debug)

.line
 *(.line)

.debug_srcinfo
 *(.debug_srcinfo)

.debug_sfnames
 *(.debug_sfnames)

.debug_aranges  0x00000000      0x160
 *(.debug_aranges)
 .debug_aranges
                0x00000000       0x20 main.o
 .debug_aranges
                0x00000020       0x20 share.o
 .debug_aranges
                0x00000040       0x20 menu.o
 .debug_aranges
                0x00000060       0x20 ./libfontprn.a(fontprn.o)
 .debug_aranges
                0x00000080       0x20 ./libbg_rsm.a(bgmain.o)
 .debug_aranges
                0x000000a0       0x20 ./libbmpmode.a(bitmap.o)
 .debug_aranges
                0x000000c0       0x20 ./libcoleffsm.a(c_effect.o)
 .debug_aranges
                0x000000e0       0x20 ./libalphasm.a(alpha.o)
 .debug_aranges
                0x00000100       0x20 ./libobj_rsm.a(obmain.o)
 .debug_aranges
                0x00000120       0x20 ./libswinsm.a(window.o)
 .debug_aranges
                0x00000140       0x20 C:\PROGRA~1\CYGNUS\THUMBELF-000512\H-I686-CYGWIN32\BIN/../lib/gcc-lib/thumb-elf/2.9-arm-000512/../../../../thumb-elf/lib/libg.a(memcpy.o)

.debug_pubnames
                0x00000000      0xe8e
 *(.debug_pubnames)
 .debug_pubnames
                0x00000000       0x1e main.o
 .debug_pubnames
                0x0000001e      0x17d share.o
 .debug_pubnames
                0x0000019b       0x8e menu.o
 .debug_pubnames
                0x00000229       0x1c menuitem.o
 .debug_pubnames
                0x00000245       0xc6 ./libfontprn.a(fontprn.o)
 .debug_pubnames
                0x0000030b      0x118 ./libbg_rsm.a(bgmain.o)
 .debug_pubnames
                0x00000423       0x4a ./libbg_rsm.a(bgexpl.o)
 .debug_pubnames
                0x0000046d       0x37 ./libbg_rsm.a(bg_map_map.o)
 .debug_pubnames
                0x000004a4       0x31 ./libbg_rsm.a(ball.o)
 .debug_pubnames
                0x000004d5       0x35 ./libbg_rsm.a(bg_map.o)
 .debug_pubnames
                0x0000050a       0x40 ./libbg_rsm.a(cl0.o)
 .debug_pubnames
                0x0000054a       0xa8 ./libbmpmode.a(bitmap.o)
 .debug_pubnames
                0x000005f2       0x4a ./libbmpmode.a(bmexpl.o)
 .debug_pubnames
                0x0000063c       0x29 ./libbmpmode.a(img24bit.o)
 .debug_pubnames
                0x00000665       0x2a ./libbmpmode.a(img24bit2.o)
 .debug_pubnames
                0x0000068f       0x38 ./libbmpmode.a(umiB.o)
 .debug_pubnames
                0x000006c7       0xc9 ./libcoleffsm.a(c_effect.o)
 .debug_pubnames
                0x00000790       0x4e ./libcoleffsm.a(ce_data.o)
 .debug_pubnames
                0x000007de       0x4a ./libcoleffsm.a(ceexpl.o)
 .debug_pubnames
                0x00000828       0x3d ./libcoleffsm.a(ce_PS_hey5.o)
 .debug_pubnames
                0x00000865       0x49 ./libcoleffsm.a(ce_bg1.o)
 .debug_pubnames
                0x000008ae       0x49 ./libcoleffsm.a(ce_bg3.o)
 .debug_pubnames
                0x000008f7       0xbf ./libalphasm.a(alpha.o)
 .debug_pubnames
                0x000009b6       0x3e ./libalphasm.a(alpha_data.o)
 .debug_pubnames
                0x000009f4       0x4a ./libalphasm.a(alexpl.o)
 .debug_pubnames
                0x00000a3e       0x49 ./libalphasm.a(ap_bg0.o)
 .debug_pubnames
                0x00000a87       0x49 ./libalphasm.a(ap_bg1.o)
 .debug_pubnames
                0x00000ad0       0x49 ./libalphasm.a(ap_bg2.o)
 .debug_pubnames
                0x00000b19       0x3d ./libalphasm.a(ap_PS_hey5.o)
 .debug_pubnames
                0x00000b56       0x91 ./libobj_rsm.a(obmain.o)
 .debug_pubnames
                0x00000be7       0x4a ./libobj_rsm.a(obexpl.o)
 .debug_pubnames
                0x00000c31       0x31 ./libobj_rsm.a(hey2.o)
 .debug_pubnames
                0x00000c62       0x64 ./libswinsm.a(window.o)
 .debug_pubnames
                0x00000cc6       0x4a ./libswinsm.a(swexpl.o)
 .debug_pubnames
                0x00000d10       0x49 ./libswinsm.a(sw_bg1.o)
 .debug_pubnames
                0x00000d59       0x49 ./libswinsm.a(sw_bg2.o)
 .debug_pubnames
                0x00000da2       0x49 ./libswinsm.a(sw_bg3.o)
 .debug_pubnames
                0x00000deb       0x49 ./libswinsm.a(sw_bg0.o)
 .debug_pubnames
                0x00000e34       0x3d ./libswinsm.a(sw_PS_hey5.o)
 .debug_pubnames
                0x00000e71       0x1d C:\PROGRA~1\CYGNUS\THUMBELF-000512\H-I686-CYGWIN32\BIN/../lib/gcc-lib/thumb-elf/2.9-arm-000512/../../../../thumb-elf/lib/libg.a(memcpy.o)

.debug_info     0x00000000    0x6b014
 *(.debug_info)
 .debug_info    0x00000000     0x2e9a main.o
 .debug_info    0x00002e9a     0x3280 share.o
 .debug_info    0x0000611a     0x3211 menu.o
 .debug_info    0x0000932b     0x2fee menuitem.o
 .debug_info    0x0000c319     0x349c ./libfontprn.a(fontprn.o)
 .debug_info    0x0000f7b5     0x333b ./libbg_rsm.a(bgmain.o)
 .debug_info    0x00012af0     0x2e40 ./libbg_rsm.a(bgexpl.o)
 .debug_info    0x00015930     0x274f ./libbg_rsm.a(bg_map_map.o)
 .debug_info    0x0001807f     0x2759 ./libbg_rsm.a(ball.o)
 .debug_info    0x0001a7d8     0x275e ./libbg_rsm.a(bg_map.o)
 .debug_info    0x0001cf36     0x2783 ./libbg_rsm.a(cl0.o)
 .debug_info    0x0001f6b9     0x3171 ./libbmpmode.a(bitmap.o)
 .debug_info    0x0002282a     0x2e41 ./libbmpmode.a(bmexpl.o)
 .debug_info    0x0002566b     0x2736 ./libbmpmode.a(img24bit.o)
 .debug_info    0x00027da1     0x2738 ./libbmpmode.a(img24bit2.o)
 .debug_info    0x0002a4d9     0x2761 ./libbmpmode.a(umiB.o)
 .debug_info    0x0002cc3a     0x33aa ./libcoleffsm.a(c_effect.o)
 .debug_info    0x0002ffe4     0x2e48 ./libcoleffsm.a(ce_data.o)
 .debug_info    0x00032e2c     0x2e42 ./libcoleffsm.a(ceexpl.o)
 .debug_info    0x00035c6e     0x276d ./libcoleffsm.a(ce_PS_hey5.o)
 .debug_info    0x000383db     0x2792 ./libcoleffsm.a(ce_bg1.o)
 .debug_info    0x0003ab6d     0x2792 ./libcoleffsm.a(ce_bg3.o)
 .debug_info    0x0003d2ff     0x33a5 ./libalphasm.a(alpha.o)
 .debug_info    0x000406a4     0x2e16 ./libalphasm.a(alpha_data.o)
 .debug_info    0x000434ba     0x2e41 ./libalphasm.a(alexpl.o)
 .debug_info    0x000462fb     0x2791 ./libalphasm.a(ap_bg0.o)
 .debug_info    0x00048a8c     0x2791 ./libalphasm.a(ap_bg1.o)
 .debug_info    0x0004b21d     0x2791 ./libalphasm.a(ap_bg2.o)
 .debug_info    0x0004d9ae     0x276c ./libalphasm.a(ap_PS_hey5.o)
 .debug_info    0x0005011a     0x310a ./libobj_rsm.a(obmain.o)
 .debug_info    0x00053224     0x2e41 ./libobj_rsm.a(obexpl.o)
 .debug_info    0x00056065     0x275a ./libobj_rsm.a(hey2.o)
 .debug_info    0x000587bf     0x3223 ./libswinsm.a(window.o)
 .debug_info    0x0005b9e2     0x2e40 ./libswinsm.a(swexpl.o)
 .debug_info    0x0005e822     0x278f ./libswinsm.a(sw_bg1.o)
 .debug_info    0x00060fb1     0x278f ./libswinsm.a(sw_bg2.o)
 .debug_info    0x00063740     0x278f ./libswinsm.a(sw_bg3.o)
 .debug_info    0x00065ecf     0x278f ./libswinsm.a(sw_bg0.o)
 .debug_info    0x0006865e     0x276b ./libswinsm.a(sw_PS_hey5.o)
 .debug_info    0x0006adc9      0x24b C:\PROGRA~1\CYGNUS\THUMBELF-000512\H-I686-CYGWIN32\BIN/../lib/gcc-lib/thumb-elf/2.9-arm-000512/../../../../thumb-elf/lib/libg.a(memcpy.o)

.debug_abbrev   0x00000000     0x2af3
 *(.debug_abbrev)
 .debug_abbrev  0x00000000      0x123 main.o
 .debug_abbrev  0x00000123      0x1cf share.o
 .debug_abbrev  0x000002f2      0x20a menu.o
 .debug_abbrev  0x000004fc      0x119 menuitem.o
 .debug_abbrev  0x00000615      0x1f5 ./libfontprn.a(fontprn.o)
 .debug_abbrev  0x0000080a      0x1ad ./libbg_rsm.a(bgmain.o)
 .debug_abbrev  0x000009b7      0x108 ./libbg_rsm.a(bgexpl.o)
 .debug_abbrev  0x00000abf       0xca ./libbg_rsm.a(bg_map_map.o)
 .debug_abbrev  0x00000b89       0xd1 ./libbg_rsm.a(ball.o)
 .debug_abbrev  0x00000c5a       0xca ./libbg_rsm.a(bg_map.o)
 .debug_abbrev  0x00000d24       0xe2 ./libbg_rsm.a(cl0.o)
 .debug_abbrev  0x00000e06      0x1b4 ./libbmpmode.a(bitmap.o)
 .debug_abbrev  0x00000fba      0x108 ./libbmpmode.a(bmexpl.o)
 .debug_abbrev  0x000010c2       0xca ./libbmpmode.a(img24bit.o)
 .debug_abbrev  0x0000118c       0xca ./libbmpmode.a(img24bit2.o)
 .debug_abbrev  0x00001256       0xd1 ./libbmpmode.a(umiB.o)
 .debug_abbrev  0x00001327      0x1bb ./libcoleffsm.a(c_effect.o)
 .debug_abbrev  0x000014e2      0x101 ./libcoleffsm.a(ce_data.o)
 .debug_abbrev  0x000015e3      0x108 ./libcoleffsm.a(ceexpl.o)
 .debug_abbrev  0x000016eb       0xd1 ./libcoleffsm.a(ce_PS_hey5.o)
 .debug_abbrev  0x000017bc       0xe2 ./libcoleffsm.a(ce_bg1.o)
 .debug_abbrev  0x0000189e       0xe2 ./libcoleffsm.a(ce_bg3.o)
 .debug_abbrev  0x00001980      0x179 ./libalphasm.a(alpha.o)
 .debug_abbrev  0x00001af9      0x101 ./libalphasm.a(alpha_data.o)
 .debug_abbrev  0x00001bfa      0x108 ./libalphasm.a(alexpl.o)
 .debug_abbrev  0x00001d02       0xe2 ./libalphasm.a(ap_bg0.o)
 .debug_abbrev  0x00001de4       0xe2 ./libalphasm.a(ap_bg1.o)
 .debug_abbrev  0x00001ec6       0xe2 ./libalphasm.a(ap_bg2.o)
 .debug_abbrev  0x00001fa8       0xd1 ./libalphasm.a(ap_PS_hey5.o)
 .debug_abbrev  0x00002079      0x19c ./libobj_rsm.a(obmain.o)
 .debug_abbrev  0x00002215      0x108 ./libobj_rsm.a(obexpl.o)
 .debug_abbrev  0x0000231d       0xd1 ./libobj_rsm.a(hey2.o)
 .debug_abbrev  0x000023ee      0x15d ./libswinsm.a(window.o)
 .debug_abbrev  0x0000254b      0x108 ./libswinsm.a(swexpl.o)
 .debug_abbrev  0x00002653       0xd1 ./libswinsm.a(sw_bg1.o)
 .debug_abbrev  0x00002724       0xd1 ./libswinsm.a(sw_bg2.o)
 .debug_abbrev  0x000027f5       0xd1 ./libswinsm.a(sw_bg3.o)
 .debug_abbrev  0x000028c6       0xd1 ./libswinsm.a(sw_bg0.o)
 .debug_abbrev  0x00002997       0xd1 ./libswinsm.a(sw_PS_hey5.o)
 .debug_abbrev  0x00002a68       0x8b C:\PROGRA~1\CYGNUS\THUMBELF-000512\H-I686-CYGWIN32\BIN/../lib/gcc-lib/thumb-elf/2.9-arm-000512/../../../../thumb-elf/lib/libg.a(memcpy.o)

.debug_line     0x00000000     0x28c0
 *(.debug_line)
 .debug_line    0x00000000      0x119 main.o
 .debug_line    0x00000119      0x3be share.o
 .debug_line    0x000004d7      0x501 menu.o
 .debug_line    0x000009d8      0x4b2 ./libfontprn.a(fontprn.o)
 .debug_line    0x00000e8a      0x530 ./libbg_rsm.a(bgmain.o)
 .debug_line    0x000013ba      0x300 ./libbmpmode.a(bitmap.o)
 .debug_line    0x000016ba      0x50e ./libcoleffsm.a(c_effect.o)
 .debug_line    0x00001bc8      0x467 ./libalphasm.a(alpha.o)
 .debug_line    0x0000202f      0x3f0 ./libobj_rsm.a(obmain.o)
 .debug_line    0x0000241f      0x2bc ./libswinsm.a(window.o)
 .debug_line    0x000026db      0x1e5 C:\PROGRA~1\CYGNUS\THUMBELF-000512\H-I686-CYGWIN32\BIN/../lib/gcc-lib/thumb-elf/2.9-arm-000512/../../../../thumb-elf/lib/libg.a(memcpy.o)

.debug_frame
 *(.debug_frame)

.debug_str
 *(.debug_str)

.debug_loc
 *(.debug_loc)

.debug_macinfo
 *(.debug_macinfo)

.debug_weaknames
 *(.debug_weaknames)

.debug_funcnames
 *(.debug_funcnames)

.debug_typenames
 *(.debug_typenames)

.debug_varnames
 *(.debug_varnames)

.stack          0x00080000        0x0
                0x00080000                _stack=.
 *(.stack)
OUTPUT(fncsample.elf elf32-littlearm)
